:040000008031102813
:100008007E1480312100901E0E282000901E0E289C
:100018008031C4207E10090080311228F901FA01CC
:100028007E102000172822009613642080312200B9
:100038000C152930F3009630F2007F30890B222806
:10004800F20B2228F30B22280000F40122000C15E1
:100058000530F3000F30F200F130890B3128F20B34
:100068003128F30B3128000022000C112530F30051
:100078008730F2008C30890B3F28F20B3F28F30BB6
:100088003F280A30F40A7402031C2A28CB30F300F4
:10009800EC30F2008430890B4F28F20B4F28F30B19
:1000A8004F280032E130F0000030F1005F2080314D
:1000B8009F2080315C287108F6007008F500080060
:1000C80093208031742080316F2080319B208031D3
:1000D800AC208031A02832009B019D019E010800C0
:1000E800143022008C008E01333021008C003D300A
:1000F8008E00323023008E0023308C0024008C01C7
:100108008E0125008C018E013D002108E03914384C
:10011800A1003C002408E0391038A400080032008F
:1001280091019201930194019501960108001630FE
:100138002100970008000800083023009F00903035
:100148009D0004309E0040309B0003309C00080056
:10015800473020009800E730960096309500160842
:10016800F800F7011508F704901221009016E53001
:10017800F0000030F1005F20903020009700080068
:1001880090127808960077089500F90A0319FA0A78
:1001980000307A02053003197902031C0800D720C1
:1001A800F901FA01080075087604031908007608B1
:1001B8008A0075080A0080310800043022008C0685
:0401C8000800080023
:020000040001F9
:08000E008CF750FFFFDFFFFF3C
:10E000000000000000000000000000000000000010
:10E010000000000000000000000000000000000000
:10E0200000000000000000000000000000000000F0
:10E0300000000000000000000000000000000000E0
:10E0400000000000000000000000000000000000D0
:10E0500000000000000000000000000000000000C0
:10E0600000000000000000000000000000000000B0
:10E0700000000000000000000000000000000000A0
:10E080000000000000000000000000000000000090
:10E090000000000000000000000000000000000080
:10E0A0000000000000000000000000000000000070
:10E0B0000000000000000000000000000000000060
:10E0C0000000000000000000000000000000000050
:10E0D0000000000000000000000000000000000040
:10E0E0000000000000000000000000000000000030
:10E0F0000000000000000000000000000000000020
:10E10000000000000000000000000000000000000F
:10E1100000000000000000000000000000000000FF
:10E1200000000000000000000000000000000000EF
:10E1300000000000000000000000000000000000DF
:10E1400000000000000000000000000000000000CF
:10E1500000000000000000000000000000000000BF
:10E1600000000000000000000000000000000000AF
:10E17000000000000000000000000000000000009F
:10E18000000000000000000000000000000000008F
:10E19000000000000000000000000000000000007F
:10E1A000000000000000000000000000000000006F
:10E1B000000000000000000000000000000000005F
:10E1C000000000000000000000000000000000004F
:10E1D000000000000000000000000000000000003F
:10E1E000000000000000000000000000000000002F
:10E1F000000000000000000000000000000000001F
:00000001FF
